BL51 BANKED LINKER/LOCATER V6.00                                                        01/09/2018  11:11:12  PAGE 1


BL51 BANKED LINKER/LOCATER V6.00, INVOKED BY:
C:\KEIL\C51\BIN\BL51.EXE main.obj, Delay_1T.obj TO MA82G5Dxx RAMSIZE (256)


MEMORY MODEL: SMALL


INPUT MODULES INCLUDED:
  main.obj (MAIN)
  Delay_1T.obj (DELAY_1T)
  C:\KEIL\C51\LIB\C51S.LIB (?C_STARTUP)


LINK MAP OF MODULE:  MA82G5Dxx (MAIN)


            TYPE    BASE      LENGTH    RELOCATION   SEGMENT NAME
            -----------------------------------------------------

            * * * * * * *   D A T A   M E M O R Y   * * * * * * *
            REG     0000H     0008H     ABSOLUTE     "REG BANK 0"
            DATA    0008H     0002H     UNIT         _DATA_GROUP_
            DATA    000AH     0001H     UNIT         ?DT?MAIN
            IDATA   000BH     0001H     UNIT         ?STACK

            * * * * * * *  X D A T A   M E M O R Y  * * * * * * *
            XDATA   0000H     0080H     UNIT         ?XD?MAIN

            * * * * * * *   C O D E   M E M O R Y   * * * * * * *
            CODE    0000H     0003H     ABSOLUTE     
            CODE    0003H     00A9H     UNIT         CODE_DELAY
            CODE    00ACH     003EH     UNIT         ?PR?MAIN?MAIN
            CODE    00EAH     0012H     UNIT         ?PR?_SPI_WR?MAIN
            CODE    00FCH     0010H     UNIT         ?PR?INITIAL_SPI?MAIN
            CODE    010CH     0010H     UNIT         ?PR?_SPI_RD?MAIN
            CODE    011CH     000EH     UNIT         ?PR?SPI_RD_SINGLE?MAIN
            CODE    012AH     000CH     UNIT         ?C_C51STARTUP
            CODE    0136H     000BH     UNIT         ?PR?_SPI_WR_SINGLE?MAIN



OVERLAY MAP OF MODULE:   MA82G5Dxx (MAIN)


SEGMENT                           DATA_GROUP 
  +--> CALLED SEGMENT           START    LENGTH
-----------------------------------------------
?C_C51STARTUP                   -----    -----
  +--> ?PR?MAIN?MAIN

?PR?MAIN?MAIN                   0008H    0001H
  +--> ?PR?INITIAL_SPI?MAIN
  +--> ?PR?_SPI_WR?MAIN
  +--> ?PR?_SPI_RD?MAIN

?PR?_SPI_WR?MAIN                0009H    0001H
  +--> ?PR?_SPI_WR_SINGLE?MAIN

BL51 BANKED LINKER/LOCATER V6.00                                                      01/09/2018  11:11:12  PAGE 2


?PR?_SPI_RD?MAIN                -----    -----
  +--> ?PR?_SPI_WR_SINGLE?MAIN
  +--> ?PR?SPI_RD_SINGLE?MAIN



SYMBOL TABLE OF MODULE:  MA82G5Dxx (MAIN)

  VALUE           TYPE          NAME
  ----------------------------------

  -------         MODULE        MAIN
  C:0000H         SYMBOL        _ICE_DUMMY_
  D:0091H         PUBLIC        P1M0
  D:0092H         PUBLIC        P1M1
  D:0090H         PUBLIC        P1
  D:00A0H         PUBLIC        P2
  D:00C0H         PUBLIC        XICON
  D:00B0H         PUBLIC        P3
  D:00E8H         PUBLIC        P4
  D:0085H         PUBLIC        SPCON
  D:00F8H         PUBLIC        P6
  D:00A8H         PUBLIC        IE
  D:00B8H         PUBLIC        IP0L
  C:00FCH         PUBLIC        Initial_SPI
  D:00D8H         PUBLIC        CCON
  C:00ACH         PUBLIC        main
  C:011CH         PUBLIC        SPI_RD_Single
  B:0090H.1       PUBLIC        P11
  D:0088H         PUBLIC        TCON
  B:00B0H.5       PUBLIC        P35
  C:0136H         PUBLIC        _SPI_Wr_Single
  X:0000H         PUBLIC        TestBuf
  D:000AH         PUBLIC        tmp
  D:0084H         PUBLIC        SPSTAT
  C:010CH         PUBLIC        _SPI_Rd
  D:0098H         PUBLIC        S0CON
  D:00C8H         PUBLIC        T2CON
  C:00EAH         PUBLIC        _SPI_Wr
  D:00D0H         PUBLIC        PSW
  D:0086H         PUBLIC        SPDAT
  -------         PROC          INITIAL_SPI
  C:00FCH         LINE#         14
  C:00FCH         LINE#         15
  C:00FCH         LINE#         16
  C:00FFH         LINE#         17
  C:0102H         LINE#         18
  C:0105H         LINE#         20
  C:0108H         LINE#         21
  C:010BH         LINE#         22
  -------         ENDPROC       INITIAL_SPI
  -------         PROC          _SPI_WR_SINGLE
  D:0007H         SYMBOL        Var
  C:0136H         LINE#         24
  C:0136H         LINE#         25
  C:0136H         LINE#         26
  C:0138H         LINE#         27
BL51 BANKED LINKER/LOCATER V6.00                                                      01/09/2018  11:11:12  PAGE 3


  C:013DH         LINE#         28
  C:0140H         LINE#         29
  -------         ENDPROC       _SPI_WR_SINGLE
  -------         PROC          SPI_RD_SINGLE
  -------         DO            
  D:0007H         SYMBOL        Var
  -------         ENDDO         
  C:011CH         LINE#         31
  C:011CH         LINE#         32
  C:011CH         LINE#         35
  C:011FH         LINE#         36
  C:0124H         LINE#         37
  C:0127H         LINE#         38
  C:0129H         LINE#         40
  C:0129H         LINE#         41
  -------         ENDPROC       SPI_RD_SINGLE
  -------         PROC          _SPI_WR
  D:0007H         SYMBOL        Addr
  D:0009H         SYMBOL        Dta
  C:00EAH         LINE#         43
  C:00ECH         LINE#         44
  C:00ECH         LINE#         45
  C:00EEH         LINE#         46
  C:00F1H         LINE#         47
  C:00F4H         LINE#         48
  C:00F9H         LINE#         49
  C:00FBH         LINE#         51
  -------         ENDPROC       _SPI_WR
  -------         PROC          _SPI_RD
  D:0007H         SYMBOL        Addr
  -------         DO            
  D:0007H         SYMBOL        Dta
  -------         ENDDO         
  C:010CH         LINE#         53
  C:010CH         LINE#         54
  C:010CH         LINE#         57
  C:010EH         LINE#         58
  C:0111H         LINE#         59
  C:0114H         LINE#         60
  C:0117H         LINE#         61
  C:0119H         LINE#         63
  C:011BH         LINE#         64
  C:011BH         LINE#         65
  -------         ENDPROC       _SPI_RD
  -------         PROC          MAIN
  -------         DO            
  D:0008H         SYMBOL        i
  -------         ENDDO         
  C:00ACH         LINE#         67
  C:00ACH         LINE#         68
  C:00ACH         LINE#         70
  C:00AFH         LINE#         72
  C:00AFH         LINE#         73
  C:00AFH         LINE#         74
  C:00B1H         LINE#         75
  C:00B4H         LINE#         76
  C:00B4H         LINE#         77
BL51 BANKED LINKER/LOCATER V6.00                                                      01/09/2018  11:11:12  PAGE 4


  C:00BEH         LINE#         78
  C:00C7H         LINE#         79
  C:00D1H         LINE#         80
  C:00D1H         LINE#         81
  C:00E6H         LINE#         82
  -------         ENDPROC       MAIN
  -------         ENDMOD        MAIN

  -------         MODULE        DELAY_1T
  C:0003H         SEGMENT       CODE_DELAY
  C:0084H         PUBLIC        DELAY_100US
  C:0063H         PUBLIC        DELAY_10US
  C:0046H         PUBLIC        DELAY_1US
  C:008FH         PUBLIC        DELAY_200US
  C:006EH         PUBLIC        DELAY_20US
  C:0049H         PUBLIC        DELAY_2US
  C:00A2H         PUBLIC        DELAY_500US
  C:0079H         PUBLIC        DELAY_50US
  C:0058H         PUBLIC        DELAY_5US
  C:0003H         PUBLIC        _DELAY_MS
  D:00E0H         SYMBOL        ACC
  C:002EH         SYMBOL        DELAY_UNIT_1MS
  N:0001H         SYMBOL        FOSC_12MHZ
  N:0000H         SYMBOL        FOSC_24MHZ
  C:0011H         SYMBOL        LSB_LOOP
  C:001EH         SYMBOL        MSB_LOOP0
  C:001BH         SYMBOL        MSB_LOOP1
  C:0017H         SYMBOL        NDLSB
  C:0027H         SYMBOL        NDMSB
  C:0003H         LINE#         29
  C:0005H         LINE#         30
  C:0007H         LINE#         31
  C:0009H         LINE#         33
  C:000BH         LINE#         34
  C:000DH         LINE#         36
  C:000FH         LINE#         37
  C:0011H         LINE#         39
  C:0014H         LINE#         40
  C:0017H         LINE#         42
  C:0019H         LINE#         43
  C:001BH         LINE#         45
  C:001EH         LINE#         47
  C:0021H         LINE#         48
  C:0024H         LINE#         49
  C:0027H         LINE#         51
  C:0029H         LINE#         52
  C:002BH         LINE#         53
  C:002DH         LINE#         54
  C:002EH         LINE#         57
  C:0031H         LINE#         58
  C:0034H         LINE#         59
  C:0037H         LINE#         60
  C:003AH         LINE#         61
  C:003DH         LINE#         62
  C:0040H         LINE#         63
  C:0043H         LINE#         64
  C:0044H         LINE#         65
BL51 BANKED LINKER/LOCATER V6.00                                                      01/09/2018  11:11:12  PAGE 5


  C:0045H         LINE#         66
  C:0046H         LINE#         78
  C:0047H         LINE#         78
  C:0048H         LINE#         79
  C:0049H         LINE#         91
  C:004AH         LINE#         91
  C:004BH         LINE#         91
  C:004CH         LINE#         91
  C:004DH         LINE#         91
  C:004EH         LINE#         91
  C:004FH         LINE#         91
  C:0050H         LINE#         91
  C:0051H         LINE#         91
  C:0052H         LINE#         91
  C:0053H         LINE#         91
  C:0054H         LINE#         91
  C:0055H         LINE#         91
  C:0056H         LINE#         91
  C:0057H         LINE#         92
  C:0058H         LINE#         108
  C:005AH         LINE#         109
  C:005DH         LINE#         110
  C:0060H         LINE#         111
  C:0062H         LINE#         112
  C:0063H         LINE#         127
  C:0065H         LINE#         128
  C:0068H         LINE#         129
  C:006BH         LINE#         130
  C:006DH         LINE#         131
  C:006EH         LINE#         146
  C:0070H         LINE#         147
  C:0073H         LINE#         148
  C:0076H         LINE#         149
  C:0078H         LINE#         150
  C:0079H         LINE#         165
  C:007BH         LINE#         166
  C:007EH         LINE#         167
  C:0081H         LINE#         168
  C:0083H         LINE#         169
  C:0084H         LINE#         184
  C:0086H         LINE#         185
  C:0089H         LINE#         186
  C:008CH         LINE#         187
  C:008EH         LINE#         188
  C:008FH         LINE#         206
  C:0091H         LINE#         207
  C:0094H         LINE#         208
  C:0097H         LINE#         209
  C:009AH         LINE#         210
  C:009DH         LINE#         211
  C:009FH         LINE#         212
  C:00A0H         LINE#         212
  C:00A1H         LINE#         213
  C:00A2H         LINE#         234
  C:00A5H         LINE#         235
  C:00A8H         LINE#         236
  C:00ABH         LINE#         237
BL51 BANKED LINKER/LOCATER V6.00                                                      01/09/2018  11:11:12  PAGE 6


  -------         ENDMOD        DELAY_1T

Program Size: data=12.0 xdata=128 code=321
LINK/LOCATE RUN COMPLETE.  0 WARNING(S),  0 ERROR(S)
